:100000004C29A0007F39201B803C0920A01B003C0C
:1000100008008A01820700340334063409340C34A2
:1000200010341334163419341C341F34223425345C
:1000300028342B342E3431343334363439343C3490
:100040003F3441344434473449344C344E345134D1
:100050005334553458345A345C345E34603462342A
:100060006434663468346A346B346D346F3470349D
:1000700071347334743475347634783479347A3432
:100080007A347B347C347D347D347E347E347E34EB
:100090007F347F347F347F349620B4000408B60068
:1000A0000800A4002508A402031CA5032708A60233
:1000B000031CA7033709A2003509A300A20A0319EC
:1000C000A30A4130A900AC01AD01AE01AF01A80106
:1000D0003608840034099320841348212408AC078F
:1000E0000318AD0A2508AD072608AE070318AF0AA6
:1000F0002708AF072D080120803EA1002F0801200E
:10010000803EA107210CA80700083404031C340614
:100110008000290303194130A9000319A20A031919
:10012000A30F6D284729841780054729A8000530AB
:10013000A8190530840000308A0028080739820792
:100140000134023404340834103420344034803410
:100150000F39A00083161F088F3930389F00831293
:100160000310A00DA00D1F08C139200401389F0005
:100170000030A1003230E3209F149F18BD281E08D4
:10018000A10083161E08472983169B001C141A0819
:10019000472983169A001C1555309D00AA309D00F2
:1001A0009C149C18D1281C114729A301A200FF30E0
:1001B000A207031CA307031C47290330A100E63054
:1001C000E320D728A101FC3EA000A109031CEE28D2
:1001D000FF300000A0070318E928A0076400A10F62
:1001E000E82808000310A00DA10DFF3E0318F22817
:1001F000200847290310A10CA00CFF3E0318FA2881
:1002000020084729A101A301A20002301629A1015B
:10021000A301A20003301629A20001301629A10172
:10022000A301A20006301629A2000530A800230869
:100230002102031D1D292208200204300318013069
:10024000031902302805031DFF3047290038031D1C
:10025000FF300405031DFF3047290404031DFF3050
:1002600047291030A800A101A001A70CA60C031C6F
:100270003F292208A00723080318230FA107A10C78
:10028000A00CA50CA40CA80B35292408472983131E
:10029000031383126400080089309F00EA01FF30D5
:1002A000B800DE01DF010230A820DA002108DB00FF
:1002B000DC01DD015A08A0005B08A100A301253084
:1002C0001121031D642967210A30D52053295A08BA
:1002D000A0005B08A1000330A30092300C21E000D5
:1002E0005A08A0005B08A1000330A300FF301121D1
:1002F000E2006008840062082621E200E300640056
:1003000062086304031988290130E600312473234D
:100310005A08A0005B08A1000330A30049300C215B
:10032000E0005A08A0005B08A1000330A30092304F
:100330001121E2006008840062082621E200E30047
:100340006400620863040319A9290230E60031241D
:1003500073235A08A0005B08A1000230A300FF30FD
:100360000C21E0005A08A0005B08A1000330A300A4
:1003700049301121E2006008840062082621E20071
:10038000E3006400620863040319CA290330E6002D
:10039000312473235A08A0005B08A1000230A30097
:1003A000B6300C21E0005A08A0005B08A100023022
:1003B000A300FF301121E2006008840062082621BA
:1003C000E200E3006400620863040319EB290430CF
:1003D000E600312473235A08A0005B08A100023014
:1003E000A3006D300C21E0005A08A0005B08A100BA
:1003F0000230A300B6301121E200600884006208D8
:100400002621E200E30064006208630403190C2A59
:100410000530E600312473235A08A0005B08A100D0
:100420000230A30025300C21E0005A08A0005B0830
:10043000A1000230A3006D301121E20060088400A9
:1004400062082621E200E3006400620863040319E5
:100450002D2A0630E600312473235A08A0005B08D9
:10046000A1000130A300DB300C21E0005A08A000FD
:100470005B08A1000230A30025301121E2006008D2
:10048000840062082621E200E3006400620863043D
:1004900003194E2A0730E600312473235A08A000BE
:1004A0005B08A1000130A30091300C21E0005A0844
:1004B000A0005B08A1000130A300DB301121E200A5
:1004C0006008840062082621E200E30064006208FC
:1004D000630403196F2A0830E600312473235A0895
:1004E000A0005B08A1000130A30049300C21E0000E
:1004F0005A08A0005B08A1000130A300913011212F
:10050000E2006008840062082621E200E300640043
:10051000620863040319902A0930E600312473232A
:100520005A08A0005B08A1000130A30000300C2194
:10053000E0005A08A0005B08A1000130A300493088
:100540001121E2006008840062082621E200E30035
:100550006400620863040319B12A0A30E6003124FA
:1005600073235A08A0005B08A100A301B6300C2138
:10057000E0005A08A0005B08A1000130A300003091
:100580001121E2006008840062082621E200E300F5
:100590006400620863040319D12A0B30E600312499
:1005A00073235A08A0005B08A100A3016E300C2140
:1005B000E0005A08A0005B08A100A301B630112199
:1005C000E2006008840062082621E200E300640083
:1005D000620863040319F02A0C30E6003124732307
:1005E0005A08A0005B08A100A30125300C21E000FF
:1005F0005A08A0005B08A100A3016E301121E2009F
:100600006008840062082621E200E30064006208BA
:10061000630403190F2B0D30E600312473230230DD
:10062000A820DA002108DB00DC0A0319DD0A5C08D7
:10063000A0005D08A100A30164300C21E0005A086D
:10064000A0005B08A100A30125300C21E200600896
:10065000840062082621E200E3005A08A0005B083B
:10066000A100A3016E301121E4006208630484003C
:1006700064082621E400E5006400640865040319A9
:10068000422BAB255E08A0005F08A100A30100304B
:100690001421031D672B5C08A0005D08A100A301C5
:1006A000C8300C21E0005A08A0005B08A100A3019B
:1006B0006E300C21E2006008840062082621E2000E
:1006C000E3006400620863040319672B98230A306F
:1006D000D5205A08A0005B08A100A30125300C21F9
:1006E000031D0F2B08006A08A00020300221E00043
:1006F0005E08A0005F08A100A30101300421E20010
:100700006008840062082D21E200E30064006208B2
:10071000630403198C2B08006A08383E84006608BD
:100720008000EA0A6A08383E8400FF308000080032
:1007300000304C204B30B700B5010630A700A500B3
:10074000A430A6005120640020306A020318B42BA4
:10075000FF306A07E000FF300318013EE100600847
:10076000383E8400FF308000EA01640007306602F2
:100770000318CA2BFF306607E000FF300318013E64
:10078000E1002130A600A7016008A2006108A300D3
:100790003121ED006608A00007300721E00066085F
:1007A000A0000C300F21E2006008840062082621BE
:1007B000E200E3006400620863040319EF2BF930E0
:1007C0006607E000FF300318013EE1002130A6007B
:1007D000A7016008A2006108A3003121ED006A08AA
:1007E000383E84000008E00064006008FF3C031D00
:1007F000222C0F30E700F9256D0883169B00831229
:100800006708C920EA01FF30B80000304C20E8300A
:10081000B7000330B5000530A700A500DC30A60006
:1008200051200230A820DA002108DB000A30D52050
:100830005A08A0005B08A100A30125300C21031D6C
:10084000112C08006A08383E84000008E700F925EA
:100850006D0883169B0083126708C920EA0AED0A17
:10086000EF2B5E08A0005F08A100A3010030142157
:10087000031D3B2C912C6608A00001300721E000ED
:100880006608A00006300F21E200600884006208BC
:100890002621E200E3006400620863040319602C6F
:1008A000FF306607E000FF300318013EE100213011
:1008B000A600A7016008A2006108A3003121EB0097
:1008C0006608A00007300721E0006608A0000C3091
:1008D0000F21E2006008840062082621E200E300A4
:1008E0006400620863040319852CF9306607E00090
:1008F000FF300318013EE1002130A600A701600887
:10090000A2006108A3003121EB0064000D306602F3
:10091000031C8B2C08006608E8006B08C420E70065
:100920001526640066080F3C031D972C0800640020
:100930006608013C031DA92C00304C204B30B70049
:10094000B5018430A6000330A7000230A500BC30FA
:10095000512064006608023C031DBB2C00304C2073
:100960004B30B700B5014C30A6000430A700023070
:10097000A500BC30512064006608033C031DCD2C4B
:1009800000304C204B30B700B5014C30A60004308D
:10099000A7000330A5008430512064006608043CA1
:1009A000031DDF2C00304C204B30B700B501143054
:1009B000A6000530A7000230A500BC30512064001D
:1009C0006608053C031DF12C00304C204B30B7006D
:1009D000B5011430A6000530A7000330A50084300F
:1009E000512064006608063C031D032D00304C2096
:1009F0004B30B700B5011430A6000530A700043015
:100A0000A5004C30512064006608073C031D152DDD
:100A100000304C204B30B700B501DC30A60005306B
:100A2000A7000230A500BC30512064006608083CD5
:100A3000031D272D00304C204B30B700B501DC30B2
:100A4000A6000530A7000330A500843051206400C3
:100A50006608093C031D392D00304C204B30B7008F
:100A6000B501DC30A6000530A7000430A5004C30ED
:100A70005120640066080A3C031D4B2D00304C20B9
:100A80007830B700B501A430A6000630A7000430C6
:100A9000A5004C305120640066080B3C031D5D2D01
:100AA00000304C204B30B700B501DC30A6000530DB
:100AB000A7000530A50014305120640066080C3CE6
:100AC000031D6F2D00304C204B30B700B501A43012
:100AD000A6000630A7000530A500DC3051206400D8
:100AE00066080D3C031D802D00304C20E830B70017
:100AF0000330B5000A30A700A5002830A600512019
:100B00006608A0000D300221E0005E08A0005F082A
:100B1000A100A30101300421E20060088400620802
:100B20002621E200E30064006208630403199C2D9F
:100B30000530A300DC30D6205E08A0005F08A100CD
:100B4000A30100301421031DA62D0800EB0A4B3031
:100B5000D5208D2C08005E08A0005F08A100A3012D
:100B600001301421031DD02DDE01DF01DC01DD0188
:100B700000304C204B30B700B5010630A700A5006F
:100B8000A430A600512000304C204B30B700B501F6
:100B90000530A700A5001430A60051200800F82D4C
:100BA0005E08A0005F08A100A30100301421031D0E
:100BB000F82D0130DE00DF01DC01DD0100304C20CA
:100BC0004B30B700B5010530A700A5001430A600D2
:100BD000512000304C204B30B700B5010630A70043
:100BE000A500A430A6005120EA01FF30B80008009B
:100BF0000800640007306602031C062E0F30E9006F
:100C00006708A000A1010430F520E7006400073068
:100C1000660203180D2EF030E9006D08C420EC00C8
:100C20006908EC056C08E70408006808A0000730B4
:100C30000721E0006808A0000C300F21E2006008E6
:100C4000840062082621E200E30064006208630475
:100C50000319312E6708A000A1010430FD20E60031
:100C60004B2E6808A00001300721E0006808A000B2
:100C700006300F21E2006008840062082621E200AD
:100C8000E30064006208630403194B2E0F30E9008F
:080C900067086905E600080091
:02400E00EA3096
:00000001FF
